:1000000000308B0010308500003086008316C13030
:10001000810018308500F03086008312861B83290A
:100020008515051485140A309800990096019701EA
:1000300090019611AA20B620B320CC201D214F217B
:100040006F202C206F202C2033209F0D9F1E1A28FC
:100050009F0103101F141A28DF30930000000000D6
:10006000930B2E28080083168511831285118611A3
:100070000000000000000000000000000000000080
:10008000000000000000810183168515831286158B
:10009000851D48280108A3009D00811E4D280430BD
:1000A0002302031CFC30043EA30023185E28A30C8B
:1000B000A313971A1717971E17136528A30CA313DA
:1000C000971A1713971E1717000000000000000072
:1000D0009830930000000000930B6A28080003305A
:1000E0008A00100800238A019A0008309400051144
:1000F0009A0DA420031C05159E200515A420940B21
:1001000077280511A420971E05159E200515A4200B
:100110000511A420171F05159E200515A420110800
:100120009A000830940005119A0DA420031C0515AF
:100130009E200515A420940B9328080021309300DD
:100140000000930BA0280800043093000000930BDC
:10015000A62808001808860005100514190886004E
:1001600085108514080023089E0008009B010430B8
:100170009C0086010314860D0310061ACB289B0AE7
:10018000861ACB289B0A061BCB289B0A861BCB28EA
:100190009B0A9C0BBB2808001B1A192901308A00F6
:1001A0001B08E0219B000A301B020318EB281619DC
:1001B00008001618E328161496141B0898000A3035
:1001C0009900692108009618080016101B0899006C
:1001D00016155221080096191A2996150A301B0285
:1001E000031DF62801309E0097061A290B301B02CA
:1001F000031DFD28203097061A290C301B02031D11
:100200000429023097061A290D301B02031D0B2901
:10021000043097061A290E301B02031D12290830DC
:1002200097061A290F301B02031D1A291030970652
:100230001A299611961016110800961D26290A30C3
:100240001B02031D2629C03091000800A0010310E5
:100250001F1C2E29171C2E291030A0009F1C34298A
:10026000203097186030A0001F1D3A293030171930
:100270007030A0009F1D4029403097198030A000A9
:100280001F1E46295030171A9030A0001E08A007E4
:1002900002308A00200800228A0191000800051A15
:1002A0004F2908001808A1000310210DA10EA10C70
:1002B0002107190790004030100203186729100821
:1002C0008900831608148312080897000800970114
:1002D00008004030100203180800100889001708B1
:1002E000880083168B130812881108155530890071
:1002F000AA30890088140811831208008316881810
:100300007F2983120800332098010A309D02031CC4
:0E0310008B29980A86291D079900AA208329A7
:1003C00082070134023403340F3404340534063414
:1003D0000E340734083409340D340A3400340B3435
:0203E0000C34DB
:100400008207113491343134B13419349934393488
:10041000B934123492343234B2341A349A343A340D
:10042000BA344534C5346534E5344D34CD346D3497
:10043000ED344634C6346634E6344E34CE346E344D
:10044000EE345034D0347034E4345834D834783402
:10045000F8345234D2347234F2345A34DA347A34CE
:10046000FA34043484342434A4344C348C342C349E
:10047000AC34063486342634A6340E348E342E340E
:10048000AE34143494343434B4341C349C346C346A
:10049000BC34163496343634B6341E349E343E346E
:1004A000BE345434D4347434F4345C34DC347C34AA
:1004B000EC345634D6347634F6345E34DE347E345E
:1004C000FE345134D1347134F1345934D93479345F
:1004D000F9345334D3347334B3345B34DB347B3486
:1004E000FB34053485342534A5340D348D342D3456
:1004F000AD34073487342734A7341B348F342F347A
:10050000AF34153495343534B5341D349D343D3411
:10051000BD34173497343734B7341F349F343B34E9
:10052000BF345534D5347534F5345D34DD347D3421
:10053000FD345734D7347734F7345F34DF347F34C5
:02054000BB34CA
:100600008207AA34C03480343034F034B03420341B
:10061000E034A0340C34CC348C343C34FC34BC3462
:100620002C34EC34AC340834C83488343834F834DE
:10063000B8342834E834A8340334C334833433342E
:10064000F334B3342334E334A3340F34CF348F344E
:100650003F34FF34BF342F34EF34AF340B34CB345A
:100660008B343B34FB34BB342B34EB34AB340234AB
:10067000C23482343234F234B2342234E234A2341A
:100680000E34CE348E343E34FE34BE342E34EE344A
:10069000AE340A34CA348A343A34FA34BA342A3496
:1006A000EA34003440346034973470344834683469
:1006B0005834783444346434543474344C346C34A2
:1006C0005C347C3442346234523472344A346A3496
:1006D0005A347A3446346634563476344E346E3472
:0206E0005E3486
:02400E00F93F78
:1042000000000000000000000000000000000000AE
:10421000000000000000000000000000000000009E
:10422000000000000000000000000000000000008E
:10423000000000000000000000000000000000007E
:10424000000000000000000000000000000000006E
:10425000000000000000000000000000000000005E
:10426000000000000000000000000000000000004E
:10427000000000000000000000000000000000003E
:00000001FF
